:020000040000FA
:10040000BFFFDFFFFFFFFFFFFFFFFFFFFFFFFFFF5C
:10041000FFFFFFFFFFFFFFFFFFFFFFFFFFFFFFFFEC
:10042000FFFFFFFFFFFFFFFFFFFFFFFFFFFFFFFFDC
:10043000FFFFFFFFFFFFFFFFFFFFFFFFFFFFFFFFCC
:10044000FFFFFFFFFFFFFFFFFFFFFFFFFFFFFFFFBC
:10045000FFFFFFFFFFFFFFFFFFFFFFFFFFFFFFFFAC
:020000040000FA
:10800000500D0020258300002D8300002F830000E9
:10801000318300003383000035830000000000003E
:108020000000000000000000000000006582000069
:108030003983000000000000C18200002597000085
:10804000ED8B0000FD8B00000D8C00001D8C0000EE
:108050002D8C00003D8C00004D8C00005D8C0000DC
:108060006D8C00007D8C00008D8C00009D8C0000CC
:10807000AD8C0000BD8C0000CD8C0000DD8C0000BC
:1080800075880000898800003F8300003F8300005E
:108090003F8300003F8300003F8300003F830000D8
:1080A000BD880000D3880000E9880000FF88000038
:1080B000158900003F890000558900003F830000BA
:1080C0003F8300003F8300003F8300003F830000A8
:1080D0003F8300003F8300003F8300003F83000098
:1080E0003F8300003F8300003F8300003F83000088
:1080F0003F8300003F8300003F8300003F83000078
:108100003F8300003F8300003F8300003F83000067
:108110003F8300003F8300003F8300003F83000057
:108120003F8300003F8300003F8300003F83000047
:108130003F8300003F8300003F8300003F83000037
:108140003F8300003F8300003F8300003F83000027
:108150003F8300003F8300003F8300003F83000017
:108160003F8300003F8300003F8300003F83000007
:108170003F8300003F8300003F8300003F830000F7
:108180003F8300003F8300003F8300003F830000E7
:108190003F8300003F8300003F8300003F830000D7
:1081A0003F8300003F8300003F8300003F830000C7
:1081B0003F8300003F8300003F8300003F830000B7
:1081C0003F8300003F8300003F8300003F830000A7
:1081D0003F8300003F8300003F8300003F83000097
:1081E0003F8300003F8300003F8300003F83000087
:1081F0003F8300003F8300003F8300003F83000077
:108200003F8300003F8300003F8300003F83000066
:108210003F8300003F830000058E00003F83000085
:10822000D58F00003F8300003F8300003F830000A4
:108230003F8300003F8300003F8300003F83000036
:108240003F8300003F8300003F8300003F83000026
:10825000DFF80CD000F0ECF800480047E5A1000082
:10826000500D00202C4B19680868B0E8F04F80F3DF
:108270000988BFF36F8F4FF0000080F311887047BB
:108280000000000008480068006880F308884FF08C
:10829000000080F3148862B661B6BFF34F8FBFF35E
:1082A0006F8F00DF00BF00BF08ED00E0DFF80C00BB
:1082B000016841F470010160704700BF88ED00E083
:1082C000EFF30980BFF36F8F134B1A681EF0100F86
:1082D00008BF20ED108A20E9F04F106009B44FF07C
:1082E000500080F31188BFF34F8FBFF36F8F03F0FF
:1082F00081FB4FF0000080F3118809BC1968086801
:10830000B0E8F04F1EF0100F08BFB0EC108A80F3F9
:108310000988BFF36F8F70471C82FF1FEFF3058042
:10832000704700000648804706480047FEE7FEE722
:10833000FEE7FEE7FEE7FEE7FEE7FEE7FEE7FEE715
:1083400025980000518200002DE9F05F05460020CD
:1083500092469B4688460646814640241BE02846B6
:1083600041464746224600F053F853465A46C01A43
:10837000914110D311461846224600F016F82D1AE6
:1083800067EB01084F4622460120002100F00DF85E
:1083900017EB00094E41201EA4F10104DFDC484622
:1083A00031462A464346BDE8F09F202A04DB203AA6
:1083B00000FA02F1002070479140C2F1200320FA38
:1083C00003F319439040704740EA01039B0703D031
:1083D00009E008C9121F08C0042AFAD203E011F804
:1083E000013B00F8013B521EF9D27047D2B201E0C6
:1083F00000F8012B491EFBD270470022F6E710B5AA
:1084000013460A4604461946FFF7F0FF204610BD02
:10841000202A04DB203A21FA02F00021704721FAD9
:1084200002F3D040C2F12002914008431946704740
:10843000064C074D06E0E06840F0010394E80700B1
:1084400098471034AC42F6D3FFF706FF9CC60000F5
:10845000BCC6000030B58C1810F8012B12F00F03C9
:1084600001D110F8013B120906D110F8012B03E0ED
:1084700010F8015B01F8015B5B1EF9D101E001F826
:10848000013B521EFBD1A142E6D3002030BD026861
:1084900061F308020260704708B50021009102E014
:1084A0000099491C009100998142F9D308BD000050
:1084B000014604480078084008B1012070470020B8
:1084C000FCE700003C40054070B50446002564B957
:1084D0001648007800F00700052801D1AD1F22E002
:1084E00001201249091D08701DE01048DA300068AB
:1084F000C0F3C01030B94FF48051082000F073F879
:10850000054605E04FF48051012000F06CF8054667
:108510004DB900200549091D08704FF480512020F5
:1085200000F061F80546284670BD00002640054071
:1085300070B5044614B96FF0020514E02079C10942
:108540000A48006861F3C71008490860606808605D
:10855000207820B90120FFF7B7FF054603E000208F
:10856000FFF7B2FF0546284670BD000000410540F8
:108570000146002009B9C01E22E000224A604A6874
:1085800022F080024A604A6822F003024A60132304
:108590004A6863F310224A604A6822F0704202F18E
:1085A00080524A604A6822F0706202F180724A602A
:1085B0004A6822F4700202F580124A6001220A70B1
:1085C000704770B504460D462946204600F0DEFF90
:1085D00001F0C2F870BD10B50446204601F040F825
:1085E00001F0BAF810BD18B503460A460020009005
:1085F0006FF0070409E01846FFF75AFF012801D180
:10860000002405E00098401C009000989042F2D9A8
:1086100000BF204618BD000070B504460025F4B91F
:108620001548007800F00700032801D1AD1F20E0B5
:108630001148DA300068C0F3C01058B90E48001D68
:10864000007810B96FF0050513E001200A490C31DC
:1086500008700EE0012008490C31087009E0002084
:1086600005490C3108704FF480510820FFF7BBFF1B
:108670000546284670BD00002640054070B50446FA
:1086800014B96FF0020514E0E0780B4908706078C7
:1086900040F08000A178084308490870207820B98C
:1086A0000120FFF7B9FF054603E00020FFF7B4FF04
:1086B0000546284670BD0000A240054050CC04404D
:1086C0000146002009B9C01E06E001220A700022FE
:1086D0008A704A700522CA7070470346012A05D184
:1086E0000120884000F03F00D86104E0012088406C
:1086F00000F03F0058630020704782690A4382619E
:10870000704701607047F0B5034600200AB9C01EEB
:1087100028E003F1400505EB811556682E6003F152
:10872000440505EB811596682E60968A156945EA21
:10873000064603F1480505EB81152E6003F15C0543
:1087400005EB8114D6681568354396693543D669BB
:10875000354341F20F363540266841F20F37BE43AC
:1087600035432560F0BD000010B5084A00210848D7
:1087700000F018F84FF480720021054800F01AF854
:10878000012200210248FFF7A8FF10BD1480FF1F3F
:1087900000300540034603F1440000EB8110026005
:1087A00000207047034603F1400000EB8110026097
:1087B0000020704710B5034603F1480000EB811418
:1087C000206862F31F402060002010BD0146002099
:1087D00009B9C01E0AE000220A604A608A60CA60C5
:1087E00001220A6100224A618A61CA617047000061
:1087F00010B502210948FFF780FF094A0121074807
:10880000FFF7C8FF0C2201210448FFF7D3FF012224
:1088100011460248FFF761FF10BD0000003005401F
:108820003885FF1F014600220F48006861F30300EE
:108830000D4B186010E0521C0C48006AC0F3026334
:108840000B480068D84044F62063B0FBF3F0904238
:1088500002D26FF0070070470348006800F00F0075
:108860008842E8D10020F6E71804014000400540A6
:108870004801002010B5012000F080F8012801D146
:1088800000F074F810BD000010B5022000F076F87A
:10889000012805D103A001F039F8022000F066F8A4
:1088A00010BD0000455854494E545F4348303120B4
:1088B000696E74657272757075740A0010B54FF444
:1088C000807000F05BF8012802D1000200F04EF841
:1088D00010BD10B54FF4007000F050F8012802D11F
:1088E000400200F043F810BD10B54FF4806000F076
:1088F00045F8012802D1800200F038F810BD10B50B
:108900004FF4006000F03AF8012802D1C00200F0F4
:108910002DF810BD10B54FF4805000F02FF801284D
:108920000CD10103042000F0CFF84FF48051022055
:1089300000F0CAF84FF4805000F018F810BD10B5E0
:108940004FF4005000F01AF8012802D1400300F063
:108950000DF810BD10B54FF4804000F00FF801285D
:1089600002D1800300F002F810BD00000249896DB9
:108970000143014A916570470010054001460448D3
:10898000406D084008B1012070470020FCE700005E
:1089900000100540012905D1054A12688243044BA5
:1089A0001A6004E0024A12680243014B1A607047E1
:1089B00000800440012905D1054A52688243044BD6
:1089C0005A6004E0024A52680243014B5A60704701
:1089D0000080044030B503460C46002115E0012517
:1089E0008D4025407DB10A4D05EB831505EB8100D7
:1089F000012A04D1058845F40045058003E0058877
:108A0000C5F30E0505804D1CE9B21029E7D330BD32
:108A1000003C05402DE9F04104460F4600200AB90C
:108A2000C01E4CE0002148E04FF0010C0CFA01FCA4
:108A30000CEA070CBCF1000F3BD0B2F800C0B2F852
:108A400002804CEA080CB2F804804CEA080CB2F838
:108A500006804CEA080CB2F80A804CEA080CB2F81E
:108A60000E804CEA080CB2F810804CEA080CB2F800
:108A700008804CEA080545F27723B2F814C04CEAA6
:108A8000050543F40043B2F812C04CEA050543F46F
:108A90008063DFF830C00CEB841C0CEB8106B6F869
:108AA00000C02CEA030C05EA03084CEA080CA6F8FF
:108AB00000C001F1010C0CF0FF011029B4D3BDE896
:108AC000F0810000003C05400246054B03EB02101C
:108AD000B0F80008084008B1012070470020FCE70A
:108AE0000030054010B5044B102404FB00321388FD
:108AF0000B43138010BD00000A38054030B5034613
:108B000000200BE0012585400D402DB1054D05EB02
:108B1000831505EB80042280451CE8B21028F1D3B0
:108B200030BD0000023C054010B5044B102404FB8E
:108B3000003213880B43138010BD00000838054035
:108B40000549098848F6FF72114000F4E0421143DC
:108B5000014A118070470000F83B054001460020A3
:108B600009B9C01E0BE000220A804A80CA808A82AE
:108B70008A810A814A81CA810A828A804A82704730
:108B800030B50146002009B9C01E2AE0B1F9023013
:108B90000F2B02DD6FF0020023E04B88114C0425FF
:108BA00015FB03421368C3F3080340F2FF14A3420A
:108BB00008D10B881360B1F902400B4D4B6845F8A2
:108BC00024300EE00B881468C4F30804A34206D1D5
:108BD000B1F90240044D4B6845F8243001E06FF0D4
:108BE000010030BD5C100540AC85FF1F10B5024987
:108BF0000868804710BD0000AC85FF1F10B5024912
:108C00004868804710BD0000AC85FF1F10B50249C1
:108C10008868804710BD0000AC85FF1F10B5024971
:108C2000C868804710BD0000AC85FF1F10B5024921
:108C30000869804710BD0000AC85FF1F10B50249D0
:108C40004869804710BD0000AC85FF1F10B5024980
:108C50008869804710BD0000AC85FF1F10B5024930
:108C6000C869804710BD0000AC85FF1F10B50249E0
:108C7000086A804710BD0000AC85FF1F10B502498F
:108C8000486A804710BD0000AC85FF1F10B502493F
:108C9000886A804710BD0000AC85FF1F10B50249EF
:108CA000C86A804710BD0000AC85FF1F10B502499F
:108CB000086B804710BD0000AC85FF1F10B502494E
:108CC000486B804710BD0000AC85FF1F10B50249FE
:108CD000886B804710BD0000AC85FF1F10B50249AE
:108CE000C86B804710BD0000AC85FF1F10B504465F
:108CF00004F0010048B100BF40F223101A49086097
:108D000043F21020086000BF00BF04F0020028B149
:108D100000BF16481649086100BF00BF04F00400F8
:108D200030B100BF4AF201501249088000BF00BFB5
:108D300004F0100018B14AF2085000F04FFB04F0A4
:108D4000400018B14AF2035000F048FB04F08000E4
:108D500040B100BF77200849086007490831086022
:108D600000BF00BF10BD0000000401400100A5A528
:108D700000800440FC3B05400408054010B5044653
:108D800004F0010028B100BF00201949086000BFAD
:108D900000BF04F0020028B100BF16481649086160
:108DA00000BF00BF04F0040030B100BF4FF4254005
:108DB0001249088000BF00BF04F0100018B14AF249
:108DC000085000F0FDFA04F0400018B14AF20350D8
:108DD00000F0F6FA04F0800040B100BF76200849A8
:108DE000086007490831086000BF00BF10BD0000DF
:108DF000000401400000A5A500800440FC3B0540A4
:108E00000408054030B59FB0002501215D4800F001
:108E1000CFFA012845D101215A4800F0A7F95AA0FC
:108E200000F074FD04AA4021564800F0C1F9002862
:108E300037D1002405E00EA8015D5AA000F066FDC0
:108E4000641C082CF7DB0598C0B28DF8000004986C
:108E5000019008208DF80100DDE90E01CDE9020145
:108E60000498B0F5F66F07D100234F4A04A94F4884
:108E7000006802F05BFF06E002234B4A69464C485B
:108E8000006802F053FF00BF4748006838B14FF058
:108E9000805048490860BFF34F8FBFF36F8F00BF0A
:108EA00000BF0421374800F083FA012803D10421D0
:108EB000344800F05BF91021324800F079FA0128BB
:108EC00045D110212F4800F051F93BA000F01EFDC4
:108ED00004AA41212B4800F06BF9002837D1002467
:108EE00005E00EA8015D2FA000F010FD641C082C09
:108EF000F7DB0598C0B28DF80000049801900820B7
:108F00008DF80100DDE90E01CDE902010498B0F50C
:108F1000F66F07D10223244A04A92448006802F00E
:108F200005FF06E00223204A69462148006802F056
:108F3000FDFE00BF1C48006838B14FF080501D494D
:108F40000860BFF34F8FBFF36F8F00BF00BF40219A
:108F50000C4800F02DFA012807D14021094800F003
:108F600005F92946074800F003F94FF400210548A8
:108F700000F01EFA012803D1C104024800F0F6F8FF
:108F80001FB030BD009002405278204649464F5FE6
:108F900030206E6577206D6573736167652D3E0DBA
:108FA0000A000000257820000C80FF1F0080FF1FB2
:108FB0000480FF1F04ED00E05278204649464F5FD1
:108FC00031206E6577206D6573736167652D3E0D89
:108FD0000A00000030B59FB000250121504800F084
:108FE000E7F9012838D101214D4800F0BFF84DA024
:108FF00000F08CFC04AA4021494800F0D9F858BB85
:10900000002405E00EA8015D4DA000F07FFC641C6B
:10901000082CF7DB0598C0B28DF800000498019089
:1090200008208DF80100DDE90E01CDE902010223DF
:10903000444A69464448006802F078FE00BF41484F
:10904000006838B14FF0805040490860BFF34F8F3F
:10905000BFF36F8F00BF00BF0421314800F0A8F9B3
:10906000012803D104212E4800F080F810212C485B
:1090700000F09EF9012838D11021294800F076F837
:1090800033A000F043FC04AA4121254800F090F8E9
:1090900058BB002405E00EA8015D29A000F036FCB5
:1090A000641C082CF7DB0598C0B28DF8000004980A
:1090B000019008208DF80100DDE90E01CDE90201E3
:1090C0000223204A69462048006802F02FFE00BFB4
:1090D0001C48006838B14FF080501C490860BFF34D
:1090E0004F8FBFF36F8F00BF00BF40210C4800F0CF
:1090F0005FF9012807D14021094800F037F82946D7
:10910000074800F035F84FF40021054800F050F909
:10911000012803D1C104024800F028F81FB030BD77
:10912000009402405278204649464F5F30206E65D9
:1091300077206D6573736167652D3E0D0A00000031
:10914000257820001080FF1F0880FF1F04ED00E03D
:109150005278204649464F5F31206E6577206D6515
:1091600073736167652D3E0D0A000000016570474D
:10917000C0F8D010704700000146AC31486C4FF683
:10918000FC731840084BC21808684FF6FC7318406F
:10919000054B1844121A0869AC39C0F30220034B7E
:1091A000185CB2FBF0F0704700B0024094C60000BB
:1091B0002DE9FC5F04460F4615464FF000080020DD
:1091C000009083466FF00209002D7CD08146402F2D
:1091D0002ED1D4F8A00000F4FE0008B96FF0020907
:1091E000B9F1000F06D1D4F8A40000F07F0008B94F
:1091F0006FF00809B9F1000F6CD1A0346068C0F3BA
:10920000052B20684FF6FC710840664900EB010809
:10921000E06900F007006449085C1BFB0088E06916
:10922000A03C00F0070008306049085C009051E065
:10923000412F2ED1D4F8B00000F4FE0008B96FF031
:109240000209B9F1000F06D1D4F8B40000F07F0094
:1092500008B96FF00809B9F1000F3BD1B03460686C
:10926000C0F3052B20684FF6FC7108404D4900EB18
:109270000108E068C0F302104B49085C1BFB008842
:10928000E068B03CC0F3021008304849085C009028
:1092900020E02046FFF770FFB84202D86FF00209C5
:1092A00018E054F8AC0F4FF6FC7108403D4900EB54
:1092B00001082069C0F302203B49085C07FB0088D5
:1092C0002069AC3C00E057E0C0F302200830374989
:1092D000085C0090B9F1000F61D146463068C0F3D8
:1092E00080706860686820B93068C0F38A40286080
:1092F00003E0306820F0604028603068C0F34070C0
:10930000A8603068C00F286108F10406308880B278
:10931000E8613068C0F30340E8602449E868085C0D
:10932000A866A96E0098814201D90098A8663068A5
:10933000C0F3005068613068C0F34050A8613068E5
:10934000C0F3066028623068C00F686208F1080642
:1093500001964FF0000A08E0019810F80A1005F194
:10936000280000F80A100AF1010AA86E5045F3D847
:10937000402F02D1C4F8A8B011E0412F02D1C4F8A7
:10938000B8B00CE0202F04D20120B840C4F89800F7
:1093900005E007F01F0101208840C4F89C00484602
:1093A000BDE8FC9F00B0024094C6000084C60000E7
:1093B00002460020136D0B4003B1012070470000EE
:1093C00004490988814341F42541034AA2F8FE1368
:1093D00070470000FE4305400040054003490988EE
:1093E0000143034AA2F8FE1370470000FE43054004
:1093F0000040054000B587B00020ADF8060001AA86
:109400004FF480610220FFF705FB07B000BD00B5F7
:1094100087B00220ADF806000420ADF8080001AACC
:1094200001020220FFF7F6FA07B000BD42698A4345
:1094300042617047012904D1426842F04002426013
:1094400003E0426822F040024260704730B50246B5
:109450006FF00200A9B38B68082B03D1CB68B3F57A
:10946000805F2ED00B68012B06D18B6823B94B6926
:109470003BB34B69022B24D0D1E9003423438C68E1
:1094800023434C6A2343CC6823430C692343536032
:109490000C8B04F470448B6A23434FF20304234083
:1094A000D4684FF20305AC432343D3600C6A4B6985
:1094B0002343CC6923430C7E04F00C0423439361C3
:1094C000002030BD012A03D143680B43436002E012
:1094D00043688B434360704701466FF0020099B1C7
:1094E00000220A604A6008228A600022CA600A617B
:1094F0004A614FF440528A614FF48062CA6100228F
:109500000A624A628A6200207047000010B505486E
:1095100001780078401C034B1870034800F006F8EF
:1095200010BD00001882FF1F00000240016070475C
:1095300010B500F0010353B1134B1B6862F3020333
:10954000114C236023461B6861F30613236000F06F
:10955000020353B10C4B1B6862F312430A4C2360A5
:1095600023461B6861F31653236000F0040353B1D4
:10957000054B1B6862F31A63034C236023461B6888
:1095800061F31E73236010BD000805402DE9FF4103
:1095900004460D4600262E48006803902C4840687B
:1095A00002902B48806801902948C06800902948A3
:1095B000007800F00700052816D101262648244926
:1095C0000860C01248608860C86022482638006A77
:1095D000C0F3026121480068C8404CF25031B0FB32
:1095E000F1F73846FEF758FF1A482638006AA043BC
:1095F00005EA040108431749263908620846006A4B
:10960000C0F3026115480068C8404CF25031B0FB0D
:10961000F1F73846FEF740FF012E17D10C490398A9
:10962000086002984860019888600098C8600948FE
:109630002638006AC0F3026108480068C8404CF24E
:109640005031B0FBF1F73846FEF726FFBDE8FF8149
:1096500000800440264005400EFAFFFF480100202C
:109660007FB5044600252B480068039029484068D0
:1096700002902848806801902648C06800902648DB
:10968000007800F00700052801D0052C16D101252F
:10969000224820490860C01248608860C8601E489F
:1096A0002638006AC0F302611D480068C8404CF2C9
:1096B0005031B0FBF1F63046FEF7EEFE164804706E
:1096C00015482638006AC0F3026115480068C84092
:1096D0004CF25031B0FBF1F63046FEF7DDFE012DC5
:1096E00017D10C4903980860029848600198886077
:1096F0000098C86008482638006AC0F3026108482C
:109700000068C8404CF25031B0FBF1F63046FEF72D
:10971000C3FE7FBD00800440264005400EFAFFFFD7
:109720004801002010B500BF502080F31188BFF31E
:109730004F8FBFF36F8F00BF02F0D6FC18B14FF010
:1097400080500449086000BF002080F3118800BFEA
:1097500010BD000004ED00E070B52B4D2D6805F044
:1097600001051DB1294D2A4E356002E0294D284ED4
:109770003560294D2D7805F00700062840D2DFE836
:1097800000F003080C11151A214D2D68234E356089
:1097900037E0234D214E356033E04FF400451F4E36
:1097A00035602EE0194D1D4E35602AE04FF400451E
:1097B0001A4E356025E0184DDA352D68C5F30722BD
:1097C000154D263DD5F800512B0F134DDA352D6878
:1097D00005F00304104D263DD5F8005105F0800535
:1097E0000DB90A4901E00A4D2968651CB1FBF5F580
:1097F000561C75435E1CB5FBF6F5084E356000E05F
:1098000000BF00BF70BD0000840601400024F400CA
:109810004C010020002D3101264005404801002068
:1098200000127A0000B50748006840F4700005494E
:109830000860FFF791FF4FF400400249803908604B
:1098400000BD000088ED00E002461068084008B145
:10985000012070470020FCE72DE9F04781460D46C6
:1098600017469A466FF0020875B36FB3D9F80C002B
:1098700000F4805616B1B6F5805F25D1002416E0BD
:10988000534601228021484600F021F88046B8F175
:10989000000F00D00DE026B9295D484600F033F8EE
:1098A00004E035F81410484600F02DF8641CBC4262
:1098B000E6D300BFB8F1000F06D153460122402184
:1098C000484600F004F880464046BDE8F087F8B509
:1098D00005460E4614460027002000900AE0009836
:1098E000984204D9581C10B16FF0070708E000989F
:1098F000401C009031462846FFF7A6FFA042EED15B
:1099000000BF3846F8BD021D118070470FB4054BEB
:1099100010B503A9044A029800F04CF810BC5DF899
:1099200014FB000001A00000A882FF1F002807DB35
:1099300000F01F0201219140024A430942F823101E
:109940007047000080E200E000280DDB00BF00BF90
:1099500000F01F02012191404209920002F1E02231
:10996000C2F8001100BF00BF7047000010B500280A
:1099700004DB0A07130E054A135406E00A07140E07
:10998000034A00F00F031B1FD45410BD00E400E095
:1099900018ED00E002E008C8121F08C1002AFAD141
:1099A00070477047002001E001C1121F002AFBD15F
:1099B000704700002DE9FF4F8DB00F460546002689
:1099C00006E025280BD0DDE90F1290476D1C761CB0
:1099D00028780028F5D111B03046BDE8F08F00247A
:1099E000A246A1460122EC4900E0044315F8013FDC
:1099F000203B02FA03F00842F7D128782A2810D039
:109A00006FF02F022878A0F13001092914D80AEB51
:109A10008A0102EB410144F0020400EB010A6D1CD3
:109A2000F0E701CF5FEA000A03D544F40054CAF11D
:109A3000000A44F002046D1C28782E2817D115F86E
:109A4000010F44F004042A280ED06FF02F0228786A
:109A5000A0F1300109290AD809EB890102EB410183
:109A600000EB01096D1CF2E757F8049B6D1C287888
:109A70006C280FD006DC4C2817D068280DD06A2837
:109A800014D104E0742810D07A280FD10DE044F4EA
:109A900000140AE044F4801401E044F440146978AE
:109AA000814202D104F580146D1C6D1C2A786E2A47
:109AB0001FD00CDC632A31D004DC002A8BD0582A5A
:109AC00011D1A3E0642A68D0692A0CD165E0732A19
:109AD0002ED004DC6F2A73D0702A04D19BE0752A43
:109AE0006FD0782A6ED01046DDE90F129047761CB1
:109AF00050E1C4F30250022806D0032809D00428FC
:109B000001CF09D0066045E101CFF117C0E900613E
:109B100040E101CF06803DE106703BE117F8040B00
:109B20008DF8000000208DF80100EB46012003E0D5
:109B300057F804BB4FF0FF3061074FF0000102D42B
:109B40000DE008F10101884649450FDA8045F8DB50
:109B50001BF808100029F4D108E008F1010188463B
:109B60008142FADB1BF808100029F6D1DDE90F234A
:109B7000AAEB08008146214600F036F9304400EB9C
:109B8000080604E0DDE90F121BF8010B9047B8F15D
:109B90000108F7D221464846F7E00A21C4F30253F0
:109BA0004FF0000B0891022B04D001CFC117032BFB
:109BB00009D00AE0FF1D27F00707F7E8020108E0D7
:109BC00032E01FE020E000B2C117042B01D140B207
:109BD000C117031E71F1000307DA4FF0000CD0EB40
:109BE0000C006CEB01012D2302E0230504D52B238F
:109BF0008DF82430012303E0E30701D02023F7E7A9
:109C0000984658E00A2110E010210EE010204FF095
:109C1000000B08900CE010214FF0000B44F00404FE
:109C20004FF00809089103E008214FF0000B08915C
:109C3000C4F30253022B04D001CF0021032B06D022
:109C400006E0FF1D27F00707F7E8020103E080B2F6
:109C5000042B00D1C0B24FF0000823072BD5702A87
:109C600007D0DDF820C08CF0100C5CEA0B0C05D09E
:109C70000EE040238DF82430012308E050EA010370
:109C800006D030238DF824308DF825200223984605
:109C9000DDF820C08CF0080C5CEA0B0C0BD150EA0C
:109CA000010301D1630706D530238DF824304FF02E
:109CB0000108A9F10109582A04D038A20B9208AA78
:109CC0000A920BE03AA2F9E75B46089AFEF73CFBE2
:109CD0000B9B9B5C0A9A521E0A92137050EA010277
:109CE000F2D10A98ADEB000000F1200B600702D51D
:109CF00024F4803401E04FF00109D94502DDA9EBDD
:109D00000B0000E0002000EB0B0141440890AAEB9F
:109D1000010AE00306D4DDE90F232146504600F096
:109D200063F806444FF0000908E009A911F809009A
:109D3000DDE90F12904709F10109761CC145F4DBFA
:109D4000E0030CD5DDE90F232146504600F04CF826
:109D5000064404E0DDE90F1230209047761C089994
:109D6000481E08900029F5DC08E00A980A99007856
:109D7000491C0A91DDE90F129047761CBBF10001E6
:109D8000ABF1010BF1DC21465046DDE90F2300F079
:109D900019F806446D1C1BE60928010030313233E6
:109DA0003435363738396162636465660000000017
:109DB0003031323334353637383941424344454601
:109DC000000000002DE9F041044600251E4617461C
:109DD000880404D405E039462020B0476D1C641E79
:109DE000F9D52846BDE8F0812DE9F041044600256B
:109DF0001E469046C80301D5302700E0202788047E
:109E000004D505E041463846B0476D1C641EF9D5BF
:109E10002846BDE8F0810146AEE000BF00BF00BFAC
:109E200000BF00BF00BF00BF00BF00BF00BF00BF3A
:109E300000BF00BF00BF00BF00BF00BF00BF00BF2A
:109E400000BF00BF00BF00BF00BF00BF00BF00BF1A
:109E500000BF00BF00BF00BF00BF00BF00BF00BF0A
:109E600000BF00BF00BF00BF00BF00BF00BF00BFFA
:109E700000BF00BF00BF00BF00BF00BF00BF00BFEA
:109E800000BF00BF00BF00BF00BF00BF00BF00BFDA
:109E900000BF00BF00BF00BF00BF00BF00BF00BFCA
:109EA00000BF00BF00BF00BF00BF00BF00BF00BFBA
:109EB00000BF00BF00BF00BF00BF00BF00BF00BFAA
:109EC00000BF00BF00BF00BF00BF00BF00BF00BF9A
:109ED00000BF00BF00BF00BF00BF00BF00BF00BF8A
:109EE00000BF00BF00BF00BF00BF00BF00BF00BF7A
:109EF00000BF00BF00BF00BF00BF00BF00BF00BF6A
:109F000000BF00BF00BF00BF00BF00BF00BF00BF59
:109F100000BF00BF00BF00BF00BF00BF00BF00BF49
:109F200000BF00BF00BF00BF00BF00BF00BF00BF39
:109F300000BF00BF00BF00BF00BF00BF00BF00BF29
:109F400000BF00BF00BF00BF00BF00BF00BF00BF19
:109F500000BF00BF00BF00BF00BF00BF00BF00BF09
:109F600000BF00BF00BF00BF00BF00BF00BF00BFF9
:109F700000BF00BF4A1E91B200293FF74EAF7047A5
:109F8000012101200B4A12680AB1002011E00A4A9F
:109F900012680AB100200CE0084A12680AB10020D9
:109FA00007E0074A1368074A1268521E934200D11D
:109FB00002207047E488FF1F4082FF1F3C82FF1F82
:109FC0000C89FF1F2C82FF1F1FB5002004E04106F3
:109FD000090E0DF80010401C1028F8D3FEF7C4FB42
:109FE00014210648FFF722FA01210448FFF722FA5C
:109FF00003E04FF4FA7001F0F9FBFAE700000240C9
:10A0000013B50C46FF23012269460248FFF724FCE2
:10A0100000981CBD00D0014000B587B001A8FEF734
:10A020009DFD0220ADF806000020ADF8040001AA55
:10A030004FF480610220FEF7EDFC01AA4FF40061AD
:10A040000220FEF7E7FC4FF480610220FEF76CFD72
:10A050004FF400610220FEF767FD07B000BD70B548
:10A0600006460024FFF7C6F900251BE04FF4006107
:10A070000220FEF737FD0520FFF7CDFE4FF400610B
:10A080000220FEF751FD6006040E4FF480610220AD
:10A09000FEF71AFD08B1601CC4B20520FFF7BBFE35
:10A0A000681CC5B2082DE1DB204670BD70B50446C2
:10A0B000FFF7ADF94FF400610220FEF713FD002514
:10A0C00021E004F0800028B14FF480610220FEF707
:10A0D0002BFD04E04FF480610220FEF703FD6006D3
:10A0E000040E0520FFF797FE4FF400610220FEF7F3
:10A0F0001BFD0520FFF78FFE4FF400610220FEF7E5
:10A10000F1FC681CC5B2082DDBDB70BD10B5FFF794
:10A110007EF94FF480610220FEF706FD4FF40061E6
:10A120000220FEF701FD0520FFF775FE4FF4806168
:10A130000220FEF7D7FC0520FFF76DFE4FF400610B
:10A140000220FEF7CFFC10BD10B5FFF760F94FF409
:10A1500000610220FEF7C6FC4FF480610220FEF78A
:10A16000C1FC0520FFF757FE4FF400610220FEF707
:10A17000DBFC4FF480610220FEF7D6FC0520FFF7E0
:10A180004AFE10BD10B5C824FFF741F94FF48061B5
:10A190000220FEF7C9FC0120FFF73DFE4FF40061ED
:10A1A0000220FEF7C1FC0120FFF735FEFFF722F980
:10A1B00009E0601E84B21CB9FFF7C6FF012010BD84
:10A1C0000120FFF728FE4FF480610220FEF77CFC9F
:10A1D0000028EED14FF400610220FEF783FC00203E
:10A1E000EDE700001CB5C720FEF780FD01F05CF82C
:10A1F00000F0B4FF00F058F800F086F8C720FEF732
:10A20000BDFD0020022103460A02CDE9001017A17E
:10A210001A4801F023FF0020022103460A02CDE97B
:10A22000001017A1194801F019FF0020032103466F
:10A230004FF40072CDE9001015A1184801F00EFF8F
:10A2400001F062FB11E000BFBFF34F8F14480068BC
:10A2500000F4E06013490843001D11490860BFF392
:10A260004F8F00BF00BF00BFFDE7ECE76E636139B1
:10A270003535355F7461736B0000000049A4000040
:10A280006563363030675F7461736B00C99F00008F
:10A290006D70755F7461736B00000000D9A20000DF
:10A2A0000CED00E00000FA0500B587B001A8FEF74C
:10A2B00055FC0220ADF806000020ADF8040001AA0C
:10A2C00004210520FEF7A6FB01AA4FF4404102201D
:10A2D000FEF7A0FB07B000BD04210520FEF724FC1B
:10A2E0004FF480410220FEF71FFC4FF47A7001F01A
:10A2F0007DFA4FF480410220FEF7F4FB03E04FF4B7
:10A30000FA7001F073FAFAE710B5FFF785FE10BD99
:10A310002DE9F04107460C4615461E464FF0000851
:10A32000FFF7F4FE3846FFF7C1FEFFF72BFF80462C
:10A330002846FFF7BBFEFFF725FF8046FFF7E6FE46
:10A340002046FFF7B3FEFFF71DFF80460020FFF712
:10A3500086FE3070FFF7F8FE0020BDE8F081F8B50A
:10A3600004460E4615461F4600200090012E01DCD3
:10A37000802D00DDF8BDD6B944F001016B46022204
:10A380002046FFF7C5FF012F08D19DF8001041EAD4
:10A3900005022046022100F072F824E09DF800102A
:10A3A00021EA05022046022100F069F81BE0012E97
:10A3B00019D144F001016B4603222046FFF7A8FFA4
:10A3C000012F08D19DF8001041EA05022046032123
:10A3D00000F055F807E09DF8001021EA050220463C
:10A3E000032100F04CF800BFC4E7F8B504460D4661
:10A3F000164600200090012D01DC802E00DDF8BD06
:10A400007DB944F001016B4606222046FFF780FF2C
:10A410009DF8001021EA06022046062100F02FF8E0
:10A4200010E0012D0ED144F001016B4607222046B9
:10A43000FFF76EFF9DF8001021EA06022046072173
:10A4400000F01DF800BFDAE70F2200214020FFF7DF
:10A45000CCFF13E001230F2200214020FFF77FFFF4
:10A460004FF4FA7001F0C2F900230F221946402080
:10A47000FFF775FF4FF4FA7001F0B8F9EAE72DE93C
:10A48000F04106460C4615460127FFF73FFE3046D1
:10A49000FFF70CFEFFF776FE07462046FFF706FEA5
:10A4A000FFF770FE07462846FFF700FEFFF76AFE3B
:10A4B0000746FFF749FE0020BDE8F0812DE9F04195
:10A4C00005460E462648076826480068001D00F02D
:10A4D00049FF50B92348006890F82C1001208840AB
:10A4E00021490968814320480160681CD8B9D6B168
:10A4F0001E4948681B49096888601A4982680968CA
:10A50000CA6018490968091D8268516015490968BF
:10A51000091D8160154A134909684A611146096895
:10A52000491C11601AE07C190E4800684460BC4266
:10A5300007D20C480168091D0D48006800F036FF7D
:10A540000CE008480168091D0A48006800F02EFF69
:10A5500009480068844201D207480460BDE8F081E0
:10A560003082FF1F1C82FF1F3482FF1F0C89FF1FD8
:10A570002482FF1F2082FF1F4C82FF1F10B504465C
:10A5800000F02EFF31480068401C30490860304818
:10A59000006840B92E4804600846006801280DD1C3
:10A5A00000F054FA0AE02B48006838B928480068DF
:10A5B000C06AE16A884201D82548046026480068DC
:10A5C000401C2549086008460068606494F82C1017
:10A5D0000120884021490968084320490860E16A50
:10A5E00001EB81011E4A02EB81014868A06082688C
:10A5F000E260211D826851608160E16A01EB8101A6
:10A60000174A02EB81026261E16A01EB8101144A9F
:10A6100052F82110491CE26A02EB8202104B43F807
:10A62000221000F007FF0B48006868B10848006876
:10A63000C06AE16A884207D24FF080500949086039
:10A64000BFF34F8FBFF36F8F10BD00002C82FF1F31
:10A650001C82FF1F3882FF1F4882FF1F3482FF1FAA
:10A660003C86FF1F04ED00E010B500F0B9FE104875
:10A670000068D0B90F4800F089FE0F4800F086FE50
:10A680000C480E4908600C480D49086000220C2156
:10A690000A2001F0A9FA064908600846006820B1BE
:10A6A00008A10348006801F04BF800F0C3FE10BD9C
:10A6B0006482FF1F2089FF1F3489FF1F5C82FF1FF8
:10A6C0006082FF1F546D72510000000010B516E04B
:10A6D00000F086FE0C48C068C468201D00F042FEF1
:10A6E0000A480068401E0949086009480068401E81
:10A6F0000749086000F09EFE204600F05FF804481D
:10A7000000680028E4D110BDF888FF1F2C82FF1FCD
:10A710002882FF1F70B504460D46206C70B1216C75
:10A72000E0680144E160D4E90210884201D3216865
:10A73000E1602846226CE168FDF746FE70BD2DE918
:10A74000F04104460F4615464FF00008A66B206CFA
:10A7500048B9206800282CD1A06801F0A3FD8046EC
:10A760000020A06025E07DB93946226C6068FDF7C5
:10A770002BFE216C606808446060D4E901018842C6
:10A7800017D32068606014E03946226CE068FDF75A
:10A790001BFE216CE068411AE1602168E068884294
:10A7A00003D2216CA068411AE160022D01D106B1EB
:10A7B000761E701CA0634046BDE8F08110B50446CB
:10A7C000206B00F055FE204600F052FE10BD000048
:10A7D000002101220C4B1B68012B00D901210B4ADF
:10A7E0001268D26A0AB100200DE0094A1268012AF3
:10A7F00001D9002007E009B1002004E0054A1268F1
:10A80000054B1B68D01A70473482FF1F1C82FF1F44
:10A810003C86FF1F4C82FF1F3082FF1F0146084A03
:10A82000126812680AB9012200E000220A600A6870
:10A8300022B9034A1268D268106800E0002070470D
:10A840005C82FF1F30B54FF4F043174800F0070457
:10A850002CB1C01D20F00700134C041B1B1B02462B
:10A86000124C22600024114D6C60D018083820F082
:10A8700007000F4C206000240D4D2D686C600C4DBE
:10A880002D682C601146441A4C60094C24680C60F9
:10A89000084D4C682C60084D4C682C604FF000440B
:10A8A000064D2C6030BD00004889FF1F7082FF1FDD
:10A8B0007882FF1F8082FF1F7C82FF1F8C82FF1F18
:10A8C00000BFFFF703FF19480068012807D94FF0C0
:10A8D000805017490860BFF34F8FBFF36F8FFFF7AA
:10A8E00077FF0446022C20D301F07CF81148006861
:10A8F00011490968884201D3012000E0002050B9C5
:10A9000000BF502080F31188BFF34F8FBFF36F8FCC
:10A9100000BF00BFFEE7FFF75BFF0446022C02D337
:10A92000204600F02BFE01F0C7FDCAE73C86FF1F62
:10A9300004ED00E04C82FF1F3082FF1F2DE9F04143
:10A9400006460D4617469846069C0DB9246000E061
:10A950002760E66325640121204601F079F984F837
:10A9600050800020A064BDE8F0812DE9F05F8246B0
:10A970000F4690469B460A9E0C9C4FEA8801A522F2
:10A98000206BFDF733FDA8F10100216B01EB80097D
:10A9900029F0070909F0070008B9012000E00020AC
:10A9A00050B900BF502080F31188BFF34F8FBFF321
:10A9B0006F8F00BF00BFFEE787B1002507E0795D1C
:10A9C00004F134004155785D00B902E06D1C102D92
:10A9D000F5D300BF00214320015502E0002084F898
:10A9E0003400202E01D2012000E0002050B900BF29
:10A9F000502080F31188BFF34F8FBFF36F8F00BFDC
:10AA000000BFFEE7202E00D31F26E662E66400208A
:10AA10002065201D00F0C7FC04F1180000F0C3FC05
:10AA20002461C6F12000A06164620020606584F8A2
:10AA300058005A465146484600F07AFB20600B9871
:10AA400008B10B980460BDE8F09F000010B5002429
:10AA500007E004EB84010F4A02EB810000F096FC52
:10AA6000641C202CF5D30C4800F090FC0B4800F03F
:10AA70008DFC0B4800F08AFC0A4800F087FC0A486D
:10AA800000F084FC0448094908600448084908604B
:10AA900010BD00003C86FF1FBC88FF1FD088FF1F31
:10AAA000E488FF1FF888FF1F0C89FF1F2082FF1F0B
:10AAB0002482FF1F10B50146164800E000680368B5
:10AAC0008B42FBD30246436813448B4204D1436854
:10AAD0004C682344436001460A464B6813440468AB
:10AAE000A34211D10C4C03682468A34208D04B68E0
:10AAF0000468646823444B6003681B680B6005E0CE
:10AB0000054B1B680B6001E003680B60884200D0B6
:10AB1000016010BD7082FF1F7882FF1F2DE9F04198
:10AB200004460D4616461F464FF000086560246136
:10AB3000B5420CD8F01BA169884202D34FF001083E
:10AB400011E0211D0948006800F030FC0BE0BE4216
:10AB500004D2BD4202D34FF0010804E0211D044895
:10AB6000006800F023FC4046BDE8F0816082FF1FD2
:10AB70005C82FF1F70B5054600F032FCA86B08B977
:10AB8000012400E0002400F055FC204670BDF1B522
:10AB90000098846C002654B900BF502080F31188BF
:10ABA000BFF34F8FBFF36F8F00BF00BFFEE7A06BF7
:10ABB000E16B884201D2012000E0002050B900BFC3
:10ABC000502080F31188BFF34F8FBFF36F8F00BF0A
:10ABD00000BFFEE7A06BE16B88422CD294F9455090
:10ABE000002269462046FFF7AAFD0646681C60B9A8
:10ABF000606A08B9012000E00020D8B904F12400FF
:10AC000001F0C8FBB0B1012614E07F2D01D0012076
:10AC100000E0002050B900BF502080F31188BFF33E
:10AC20004F8FBFF36F8F00BF00BFFEE7681C40B2BD
:10AC300084F8450000BF3046F8BD000070B50546F9
:10AC40000E460E480068C068C468201D00F08AFBEC
:10AC500094F8280000F0040028B132462946204626
:10AC600000F0D6F805E094F8280000F0FE0084F823
:10AC700028002046216A884770BD00005C82FF1FC3
:10AC80007FB57FE0019800287CDB039C606908B9F0
:10AC9000012000E0002010B9201D00F063FB684691
:10ACA00000F0E2F8054601980A2869D2DFE800F0D2
:10ACB0006805072E365806082F3700BF00BF00BFB3
:10ACC00094F8280040F0010084F828000298A26956
:10ACD000811803462A462046FFF720FFA8B194F8C2
:10ACE000280000F0040038B10298A26981182A46B1
:10ACF000204600F08DF805E094F8280000F0FE00F2
:10AD000084F828002046216A88473AE000BF94F87A
:10AD1000280000F0FE0084F8280032E000BF94F81C
:10AD2000280040F0010084F828000298A061A06982
:10AD300008B1012000E0002050B900BF502080F38E
:10AD40001188BFF34F8FBFF36F8F00BF00BFFEE7C7
:10AD5000A06941192B462A462046FFF7DFFE10E086
:10AD600094F8280000F0020018B9204600F080FB9B
:10AD700005E094F8280000F0FE0084F8280000E0C8
:10AD800000BF00BF002201A90348006801F06AF873
:10AD900000287FF477AF7FBD6482FF1FF8B50546BA
:10ADA0000C4600F01FFE684600F05EF8064600986C
:10ADB00020BB44B9B54206D801F07EFB3146284697
:10ADC000FFF73CFF1CE03CB10E480068006808B982
:10ADD000012000E000200446A91B22460A48006822
:10ADE00000F0DEFC01F068FB50B94FF080500749DD
:10ADF0000860BFF34F8FBFF36F8F01E001F05CFB82
:10AE0000F8BD00006082FF1F6482FF1F04ED00E0B8
:10AE100070B504460D46164604E0A0690544204678
:10AE2000216A8847A06941192B4632462046FFF720
:10AE300075FE0028F1D170BD09480068006808B9A6
:10AE4000012000E0002020B14FF0FF3005490860EC
:10AE500005E003480068C068006802490860704760
:10AE60002082FF1F4C82FF1F70B5044601F036F9A7
:10AE7000054607480068854204D200F00BF801201F
:10AE8000206001E00020206001480560284670BD78
:10AE90006C82FF1F70B508E00D480068C068046848
:10AEA0004FF0FF312046FFF7C9FE094800680068EF
:10AEB00008B9012000E000200028EDD00448056812
:10AEC00004480068024908600248056070BD00003F
:10AED0005C82FF1F6082FF1F0E480068401C08B99B
:10AEE000012000E0002050B900BF502080F31188FD
:10AEF000BFF34F8FBFF36F8F00BF00BFFEE700BFF0
:10AF0000502080F31188BFF34F8FBFF36F8F00BFC6
:10AF100000BFFEE79082FF1F08B500BF6846FFF73D
:10AF20007DFC044620460099FFF738FFFFF7A8FE96
:10AF3000F4E770B5044600F053FA94F9455019E06F
:10AF4000A06C30B12046FFF722FE88B100F088FCEB
:10AF50000EE0606A08B9012000E0002038B904F171
:10AF6000240001F017FA18B100F07AFC00E003E0C9
:10AF7000681E45B2002DE3DC00BFFF2084F84500C9
:10AF800000F058FA00F02CFA94F9445010E02069CF
:10AF900008B9012000E0002048B904F1100001F0D8
:10AFA000F9F908B100F05CFC681E45B200E001E070
:10AFB000002DECDC00BFFF2084F8440000F03AFADA
:10AFC00070BD00002DE9F04104464FF0000800F08C
:10AFD00009FD5148006808B9FFF734FC4F48006884
:10AFE000204000287ED13CB304F10800A04223D9C0
:10AFF000083404F0070000B304F00700C0F10800B3
:10B000002044A04216D904F00700C0F1080004440F
:10B0100004F0070008B9012000E0002068B900BF73
:10B02000502080F31188BFF34F8FBFF36F8F00BFA5
:10B0300000BFFEE7002400E00024002C54D0384874
:10B040000068844250D8374E3046056801E02E46ED
:10B050002D686868A04202D228680028F7D12E48DF
:10B060000068854240D0306800F1080828683060E8
:10B070006868001B102819D92F1907F0070008B9B4
:10B08000012000E0002050B900BF502080F311885B
:10B09000BFF34F8FBFF36F8F00BF00BFFEE768683D
:10B0A000001B78606C603846FFF704FD1C49686837
:10B0B0000968081A1A490860084600681A490968A8
:10B0C000884203D216480068174908601349686827
:10B0D0000968084368600020286014480068401C24
:10B0E000124900E000E0086001F0E6F908F007000E
:10B0F00008B9012000E0002050B900BF502080F3C3
:10B100001188BFF34F8FBFF36F8F00BF00BFFEE703
:10B110004046BDE8F08100007882FF1F8C82FF1F4F
:10B120007C82FF1F7082FF1F8082FF1F8482FF1FAF
:10B13000001F4FF080730360001F21F001030360C4
:10B14000001F054B036014380260001F6FF00203FC
:10B150000360203870470000D9AE000000B595B0FC
:10B160002B2280210120FDF7C9FC28224FF4007119
:10B170000120FDF7C3FC29224FF480710120FDF767
:10B18000BDFC01218804FDF715FC0AA8FEF7A4F90F
:10B1900001200A9000200B900C900E9003200F903D
:10B1A00049F2040010904FF480601190002012903A
:10B1B00014900AA93648FEF749F901225102344891
:10B1C000FEF780F94FF4BA70ADF800000720ADF833
:10B1D0000200304801906846FDF7D2FCBDF902003C
:10B1E000FEF7A4FBBDF902000E21FEF7BFFBBDF97F
:10B1F0000200FEF7A9FB01212548FEF71BF90121FA
:10B200004FF41030FDF7C6FB02A8FDF7DFFA4FF44C
:10B210008050029001200690872007900020059022
:10B220000890042009901A4803901B48049002AA31
:10B2300001211A48FDF767FA08B100BFFEE740F2A6
:10B2400073111748FDF723F92320ADF800000620FD
:10B25000ADF80200134801906846FDF791FCBDF976
:10B260000200FEF763FBBDF902000F21FEF77EFB33
:10B27000BDF90200FEF768FB01210848FDF741FA1D
:10B28000012211460548FDF728FA15B000BD00005F
:10B29000000002400D950000AC84FF1F0030054007
:10B2A00018080140F18700000EB52C492C48FDF725
:10B2B00088F9012203210520FDF78CFB02A8FDF788
:10B2C000FFF900208DF80A0030208DF809000020D9
:10B2D0008DF8080005208DF80B0002A8FDF7CEF9C7
:10B2E0006846FDF745F900208DF8000001900198AF
:10B2F00020F0030001906321019861F31020019078
:10B30000019820F0704000F1E0400190019820F099
:10B31000706000F1E0600190019820F4700000F589
:10B32000E0000190019820F0800001906846FDF750
:10B33000FFF8002211460320FEF7FAF80122114619
:10B340000420FEF7F5F80320FDF76CFA4FF44050A7
:10B35000FDF7F6FB0520FDF73EF90EBD10221100AA
:10B360007777770701460A69D1E901309860D1E91A
:10B37000010358605068884201D1886850600020FD
:10B3800008611068401E10601068704700F10801E5
:10B3900041604FF0FF31816000F10801C16001613F
:10B3A00000210160704700210161704710B502461D
:10B3B0000B685C1C0CB9106907E002F1080000E0A2
:10B3C0004068446824689C42FAD944684C604C68E0
:10B3D000A160886041600A611468641C146010BD3B
:10B3E00000BF502080F31188BFF34F8FBFF36F8FE2
:10B3F00000BF0E480068401C0C4908600846006801
:10B40000012812D10A480068C0B208B9012000E042
:10B41000002050B900BF502080F31188BFF34F8F38
:10B42000BFF36F8F00BF00BFFEE770479082FF1F22
:10B4300004ED00E00D48006850B900BF502080F3D3
:10B440001188BFF34F8FBFF36F8F00BF00BFFEE7C0
:10B4500006480068401E054908600846006820B993
:10B46000002080F3118800BF00BF70479082FF1F4B
:10B4700070B506463546002E44D0083D2C4622497C
:10B4800060680968084008B1012000E0002050B958
:10B4900000BF502080F31188BFF34F8FBFF36F8F31
:10B4A00000BF00BFFEE7206808B9012000E00020CF
:10B4B00050B900BF502080F31188BFF34F8FBFF306
:10B4C0006F8F00BF00BFFEE70F4960680968084042
:10B4D000C0B12068B0B90C496068096888436060F1
:10B4E00000F080FA09496068096808440749086063
:10B4F0002046FFF7DFFA06480068401C0449086050
:10B5000000F0DAFF70BD00008C82FF1F7C82FF1FFD
:10B510008882FF1F154800684FF47A71B0FBF1F084
:10B5200013490860084600686FF07F41B1FBF0F0F6
:10B53000104908600D480068B0FBF0F02D21B1FB08
:10B54000F0F00D49086000204FF0E02108618861AB
:10B55000064800684FF47A71B0FBF1F0401E4FF0DE
:10B56000E021486107200861704700004801002081
:10B570009482FF1F9882FF1F9C82FF1F2DE9F041DC
:10B5800004464E480068844201D94C4804684FF094
:10B59000E020006920F001004FF0E021086108463A
:10B5A0008169601E464A126802FB00154548006822
:10B5B000854202D9434800682D1A72B6BFF34F8FF7
:10B5C000BFF36F8FFEF7DCFC80B94FF0E02080699D
:10B5D0004FF0E02148610846006940F00100086131
:10B5E00037480068401E486162B665E04FF0E020D1
:10B5F000456100204FF0E02188610846006940F075
:10B6000001000861A046B8F1000F04D0BFF34F8FCE
:10B6100030BFBFF36F8F62B6BFF34F8FBFF36F8F33
:10B6200072B6BFF34F8FBFF36F8F06204FF0E0214C
:10B6300008610846006900F48030B8B12049096803
:10B64000491E4FF0E0229269AA1A881A1D4909681A
:10B65000884203D31A490968884202D918490968FF
:10B66000481E4FF0E0214861661E12E01448006851
:10B6700060434FF0E0218969471A11480068B7FB21
:10B68000F0F6701C0E4909684843C01B4FF0E021DA
:10B69000486100204FF0E02188610846006940F0D1
:10B6A00001000861304600F07DF905480068401E41
:10B6B0004FF0E021486162B6BDE8F0819882FF1F3B
:10B6C0009482FF1F9C82FF1F70B5FCF727FE044683
:10B6D000102C16D304F1E02090F8F05315480078B0
:10B6E000854201DB012000E0002050B900BF50205E
:10B6F00080F31188BFF34F8FBFF36F8F00BF00BF80
:10B70000FEE70D48006800F4E0600C4909688842D3
:10B7100001D8012000E0002050B900BF502080F384
:10B720001188BFF34F8FBFF36F8F00BF00BFFEE7DD
:10B7300070BD0000A082FF1F0CED00E0A482FF1F7F
:10B7400030B502460B4652B900BF502484F311882D
:10B75000BFF34F8FBFF36F8F00BF00BFFEE7002125
:10B76000BBB1002012E00D4C04EBC00464689442AD
:10B7700003D10A4C04EBC0010AE031B9074C54F87C
:10B78000304014B9054C04EBC001401C0A28EAD330
:10B7900000BF09B10B604A6030BD0000EC85FF1F9F
:10B7A0002DE9F04105460E4617462C46FFF718FED8
:10B7B00094F94400401C10B9002084F8440094F926
:10B7C0004500401C10B9002084F84500FFF732FE08
:10B7D000A06B28B93A46314604F1240000F062F823
:10B7E0002046FFF7A6FBBDE8F081000070B50446D7
:10B7F0000025D4B11248006808B9012000E00020FB
:10B8000050B900BF502080F31188BFF34F8FBFF3B2
:10B810006F8F00BF00BFFEE700F0E4F80021204674
:10B82000FEF74CFE00F048FE05463DB94FF0805053
:10B8300004490860BFF34F8FBFF36F8F70BD0000E6
:10B840005882FF1F04ED00E00349096801600349C5
:10B8500009684160704700004482FF1F3082FF1F6B
:10B8600001200149086070474082FF1F70B50446FF
:10B870000D4654B900BF502080F31188BFF34F8F9D
:10B88000BFF36F8F00BF00BFFEE7054801681831A6
:10B890002046FFF78BFD01212846FEF70FFE70BD05
:10B8A0001C82FF1F70B504460E46154654B900BFF2
:10B8B000502080F31188BFF34F8FBFF36F8F00BF0D
:10B8C00000BFFEE760680F490968C8610D498268DA
:10B8D00009680A620B490968183182685160094990
:10B8E000096818318160074909688C622168491C20
:10B8F00021600DB14FF0FF3629463046FEF7DEFDE0
:10B9000070BD00001C82FF1F1CB51E4800210B46A5
:10B910008022CDE900101CA11D4800F09FFB0446C9
:10B92000012C02D100F084FE0446012C15D100BF89
:10B93000502080F31188BFF34F8FBFF36F8F00BF8C
:10B940004FF0FF30134908600120134908600020C0
:10B950001249086000F094F810E0601C08B1012062
:10B9600000E0002050B900BF502080F31188BFF3E1
:10B970004F8FBFF36F8F00BF00BFFEE7084800681E
:10B980001CBD00005082FF1F49444C4500000000D0
:10B99000C1A800004C82FF1F3882FF1F3082FF1FAA
:10B9A0005482FF1F0D49096801440D4A12689142F3
:10B9B00001D8012100E0002151B900BF502181F3DD
:10B9C0001188BFF34F8FBFF36F8F00BF00BFFEE73B
:10B9D000024909680144014A116070473082FF1F23
:10B9E0004C82FF1F02480068401C014908607047F4
:10B9F0005882FF1F1D48006818B101201C490860CB
:10BA000032E000201A4908601A480068B0FA80F055
:10BA1000C0F11F0101EB8100174A52F8200008B164
:10BA2000012000E0002050B900BF502080F31188B1
:10BA3000BFF34F8FBFF36F8F00BF00BFFEE701EB77
:10BA400081020D4B03EB820042685268426000F1B4
:10BA500008024368934202D14268526842604268D9
:10BA6000D268064B1A6000BF704700005882FF1F63
:10BA70004082FF1F3482FF1F3C86FF1F1C82FF1F76
:10BA80001CB5524800685249884201D0012000E0AC
:10BA9000002050B900BF502080F31188BFF34F8FB2
:10BAA000BFF36F8F00BF00BFFEE7484800684849FA
:10BAB000491E884201D0012000E0002050B900BF9B
:10BAC000502080F31188BFF34F8FBFF36F8F00BFFB
:10BAD00000BFFEE73F49084600780190FF200A4674
:10BAE00010700846007800909DF8000000F0F0000B
:10BAF0009DF80020904201D1012000E0002050B9C3
:10BB000000BF502080F31188BFF34F8FBFF36F8FBA
:10BB100000BF00BFFEE79DF8000000F050002E4A75
:10BB2000107007202D4A106009E02C480068401E64
:10BB30002A4A10609DF800004006000E00909DF813
:10BB4000000000F080008028EFD024480068C0F199
:10BB50000700042801D1012000E0002050B900BFF7
:10BB6000502080F31188BFF34F8FBFF36F8F00BF5A
:10BB700000BFFEE7194800680002184A106010462E
:10BB8000008800F4E0601060124A019810700F48BD
:10BB90002030006840F470000C49203108600846ED
:10BBA000006840F070400860FFF7B4FC00200C49CA
:10BBB0000860FCF77BFB0B48006840F040400949F7
:10BBC0000860FCF75FFB00201CBD000000ED00E0FA
:10BBD00071C20F4100E400E0A082FF1FA482FF1F9A
:10BBE0009082FF1F34EF00E02DE9F84305460E4632
:10BBF00017460024E5B1601EB0FBF5F0B04217D344
:10BC000005FB06F010F1550F12D805FB06F808F1F8
:10BC10005400FFF7D7F90446B4B1A14609F154091D
:10BC20003B464A46314628460094FEF787FE0BE025
:10BC300054B900BF502080F31188BFF34F8FBFF37A
:10BC40006F8F00BF00BFFEE72046BDE8F88300000D
:10BC50002DE9F04105460E4601272C4654B900BF98
:10BC6000502080F31188BFF34F8FBFF36F8F00BF59
:10BC700000BFFEE7002C42D0E06B00283FD04FF021
:10BC8000FF31E06BB1FBF0F0216C884237D3FFF756
:10BC9000A7FBD4E90F12206801FB0200A06000207E
:10BCA000A06320686060E06B401E226C216800FB8E
:10BCB0000211E160FF2084F8440084F845009EB939
:10BCC000206908B9012000E00020A8B904F11000A3
:10BCD00000F060FB80B14FF0805013490860BFF363
:10BCE0004F8FBFF36F8F07E004F11000FFF74EFB9B
:10BCF00004F12400FFF74AFBFFF79CFB00E000275C
:10BD00000FB1012000E0002050B900BF502080F3A7
:10BD10001188BFF34F8FBFF36F8F00BF00BFFEE7E7
:10BD20003846BDE8F081000004ED00E02DE9F84F51
:10BD300080468B4615461E46444654B900BF5020E7
:10BD400080F31188BFF34F8FBFF36F8F00BF00BF29
:10BD5000FEE7BBF1000F01D1206C08B9012000E023
:10BD6000002050B900BF502080F31188BFF34F8FDF
:10BD7000BFF36F8F00BF00BFFEE7022E02D1E06B62
:10BD8000012801D1012000E0002050B900BF50205F
:10BD900080F31188BFF34F8FBFF36F8F00BF00BFD9
:10BDA000FEE7FFF791FC00BF5021EFF3118081F314
:10BDB0001188BFF34F8FBFF36F8F00BF0746A06B93
:10BDC000E16B884201D3022E42D194F945A0A06BC9
:10BDD0000090324659462046FEF7B1FC0AF10100B8
:10BDE000E0B9A06C58B1022E01D1009868BB204682
:10BDF000FEF7CDFE48B345B30120286025E0606A18
:10BE000008B9012000E00020F8B904F1240000F096
:10BE1000C1FAD0B1CDB10120286016E0BAF17F0F90
:10BE200001D0012000E0002050B900BF502080F375
:10BE30001188BFF34F8FBFF36F8F00BF00BFFEE7C6
:10BE40000AF1010040B284F845004FF0010901E019
:10BE50004FF0000900BF87F3118800BF4846BDE8D6
:10BE6000F88F00002DE9F74183B005460E464FF0EC
:10BE700000082C4654B900BF502080F31188BFF34E
:10BE80004F8FBFF36F8F00BF00BFFEE70EB9206C6E
:10BE900008B9012000E0002050B900BF502080F315
:10BEA0001188BFF34F8FBFF36F8F00BF00BFFEE756
:10BEB00000F004F908B9059808B9012000E0002055
:10BEC00050B900BF502080F31188BFF34F8FBFF3EC
:10BED0006F8F00BF00BFFEE700BFFFF781FAA76BBF
:10BEE000F7B131462046FEF715FC781EA0632069A5
:10BEF00008B9012000E0002060B904F1100000F052
:10BF000049FA38B14FF080502F490860BFF34F8F86
:10BF1000BFF36F8FFFF78EFA012006B0BDE8F08106
:10BF2000059818B9FFF786FA0020F6E7B8F1000F78
:10BF300004D101A8FFF788FC4FF00108FFF77AFA57
:10BF4000FFF750FDFFF74CFA94F94400401C10B97C
:10BF5000002084F8440094F94500401C10B90020EA
:10BF600084F84500FFF766FA05A901A800F02EF84D
:10BF7000F0B92046FEF7FEFDA0B104F124000599BA
:10BF8000FFF774FC2046FEF7D4FF00F095FA002876
:10BF9000A3D14FF080500C490860BFF34F8FBFF31F
:10BFA0006F8F9AE72046FEF7C4FF00F085FA94E70A
:10BFB0002046FEF7BEFF00F07FFA2046FEF7DAFDCE
:10BFC00000288AD00020A8E704ED00E070B50546FF
:10BFD0000C4655B900BF502080F31188BFF34F8F36
:10BFE000BFF36F8F00BF00BFFEE754B900BF502002
:10BFF00080F31188BFF34F8FBFF36F8F00BF00BF77
:10C00000FEE7FFF7EDF9134802686868131A206825
:10C01000401C08B9002619E00F49286809688842C1
:10C0200006D06868904203D80126002020600DE009
:10C030002068984207D92068C01A20602846FFF778
:10C0400003FC002602E0002020600126FFF7F2F941
:10C05000304670BD3082FF1F4482FF1F2DE9FF4F25
:10C0600085B0804689461746DDE912ABB800FEF779
:10C07000A9FF064656B15C20FEF7A4FF04460CB1AA
:10C08000266304E03046FFF7F3F900E000247CB1BA
:10C090000020CDE900ABCDE902403A464946404692
:10C0A000089BFEF762FC2046FEF768FA012501E0D6
:10C0B0004FF0FF35284609B0BDE8F08F0549096803
:10C0C00009B9012005E00449096809B9022000E026
:10C0D000002070473882FF1F5882FF1F01490868FF
:10C0E000704700003082FF1F2DE9F0414FF000083B
:10C0F0006148006800287DD160480068451C5F48A1
:10C10000056015BB5E480068006808B9012000E0C2
:10C11000002050B900BF502080F31188BFF34F8F2B
:10C12000BFF36F8F00BF00BFFEE755480768554853
:10C130000068534908605348076053480068401C32
:10C1400051490860FEF778FE00BF504800688542FC
:10C1500077D300BF4A480068006808B9012000E0B2
:10C16000002020B14FF0FF304849086068E04448A3
:10C170000068C068C4686668B54202D24348066079
:10C180005EE06069D4E902128A60D4E902214A6063
:10C19000211D42688A4201D1E1684160002262614A
:10C1A0000168491E0160A06A98B1A06AD4E907122B
:10C1B0008A60D4E907214A6004F1180142688A4282
:10C1C00001D1216A41600022A2620168491E01601A
:10C1D00000BF94F82C10012088402D4909680843BD
:10C1E0002B490860E16A01EB81012A4A02EB8101D7
:10C1F000486800E037E0A0608268E260211D826844
:10C2000051608160E16A01EB8101224A02EB810207
:10C210006261E16A01EB81011E4A52F82110491C5A
:10C22000E26A02EB82021B4B43F822101A49E06AD1
:10C230000968C96A88428DD34FF001088AE700E097
:10C2400000BF15480068C06A00EB8000114951F832
:10C250002000012801D94FF001081048006808B1FA
:10C260004FF0010804E00E480068401C0C490860CB
:10C270004046BDE8F08100005882FF1F3082FF1F5A
:10C280002082FF1F2482FF1F4482FF1F4C82FF1F5A
:10C290003482FF1F3C86FF1F1C82FF1F4082FF1F4E
:10C2A0003C82FF1F70B505462C460026002D68D045
:10C2B00035480068844201D1012000E0002050B9D7
:10C2C00000BF502080F31188BFF34F8FBFF36F8FF3
:10C2D00000BF00BFFEE7206D50B900BF502080F3C3
:10C2E0001188BFF34F8FBFF36F8F00BF00BFFEE712
:10C2F000206D401E2065E16CE06A884241D0206DCF
:10C3000000283ED1201DFFF72DF840B994F82C10DD
:10C31000012088401D49096881431C480160E06C88
:10C32000E062E06AC0F12000A06194F82C100120C6
:10C33000884016490968084314490860E16A01EB1E
:10C340008101134A02EB81014868A0608268E260C3
:10C35000211D826851608160E16A01EB81010C4A14
:10C3600002EB81026261E16A01EB8101084A52F845
:10C370002110491CE26A02EB8202054B43F82210AD
:10C380000126304670BD00001C82FF1F3482FF1F53
:10C390003C86FF1F70B50646F068C46854B900BFFC
:10C3A000502080F31188BFF34F8FBFF36F8F00BF12
:10C3B00000BFFEE7A06AD4E907128A60D4E907212A
:10C3C0004A6004F1180142688A4201D1216A416041
:10C3D0000022A2620168491E0160314800680028FD
:10C3E0003FD16069D4E902128A60D4E902214A602F
:10C3F000211D42688A4201D1E168416000226261E8
:10C400000168491E016094F82C10012088402549DC
:10C410000968084323490860E16A01EB8101224A67
:10C4200002EB81014868A0608268E260211D826899
:10C4300051608160E16A01EB81011B4A02EB8102DC
:10C440006261E16A01EB8101174A52F82110491C2F
:10C45000E26A02EB8202144B43F82210FEF7ECFC76
:10C4600010E012494868E0618268226204F1180114
:10C470008268516081600D4AA26211460968491CB8
:10C48000116000BF0A49E06A0968C96A884204D994
:10C49000012501200749086000E00025284670BDFD
:10C4A0005882FF1F3482FF1F3C86FF1FE488FF1F56
:10C4B0001C82FF1F4082FF1F70B5002400265348D6
:10C4C000006850B900BF502080F31188BFF34F8F30
:10C4D000BFF36F8F00BF00BFFEE7FEF781FF4B4841
:10C4E0000068401E494908600846006800287DD160
:10C4F00047480068002879D05BE04648C068C468B7
:10C50000A06AD4E907128A60D4E907214A6004F1DD
:10C51000180142688A4201D1216A41600022A26268
:10C520000168491E01606069D4E902128A60D4E999
:10C5300002214A60211D42688A4201D1E1684160BE
:10C54000002262610168491E016094F82C100120EC
:10C5500088403149096808432F490860E16A01EBC6
:10C5600081012E4A02EB81014868A0608268E26086
:10C57000211D826851608160E16A01EB8101274AD7
:10C5800002EB81026261E16A01EB8101234A52F808
:10C590002110491CE26A02EB8202204B43F8221070
:10C5A0001F49E06A0968C96A884202D301201D490F
:10C5B00008601848006808B9012000E00020002841
:10C5C0009BD00CB1FEF738FC1748056865B100BF79
:10C5D000FFF78AFD10B10120124908606D1E002D81
:10C5E000F6D10020104908600E4800E009E000681C
:10C5F00038B1012630070D490860BFF34F8FBFF3F4
:10C600006F8FFEF717FF304670BD00005882FF1F86
:10C610002C82FF1FE488FF1F3482FF1F3C86FF1F10
:10C620001C82FF1F4082FF1F3C82FF1F04ED00E0C1
:10C630001CB50024FEF718F80D48006850B10D48ED
:10C6400002210023CA01CDE900100BA10C48FFF71D
:10C6500005FD044654B900BF502080F31188BFF394
:10C660004F8FBFF36F8F00BF00BFFEE720461CBD9A
:10C670006482FF1F6882FF1F546D7220537663002F
:10C6800019AF00000001020304050607080C10148E
:10C69000182030401014181C20283848BCC6000050
:10C6A0000080FF1FAC0200005484000008C7000097
:10C6B000AC82FF1FA48A0000A49900000115003C71
:10C6C000FF535049204D61737465722F536C61762E
:10C6D00065206578616D706C653A20436F6D6D758E
:10C6E0006E69636174696F6E206265747765656EEB
:10C6F0002074776F20626F617264732101FFA10261
:08C700003C1F0519AAAAAAAA10
:040000050000825124
:00000001FF
